:06313C0025730079490033
:10306E007BFF7A31793FC003C002C0017B007A003A
:10307E00791CA801AC02AD03D001D002D0037E00B2
:10308E007F03122D427B007A00791C122E6D8B0E5F
:10309E008A0F89107B017A007900C003C002C0013B
:1030AE007BFF7A31793C8B0B8A0C890DD001D002D3
:0530BE00D0031229728D
:0330C30080A922BF
:100003000069006E006E67006F0061006169006146
:100013006E00616E6700616F00656900656E006563
:100023006E670069616E0069616F00696500696EE2
:1000330000696E67007500650068610068616900AA
:1000430068616E0068616E670068616F00686500D3
:1000530068656E0068656E6700686900686F6E6743
:1000630000686F750068750068756169006875617F
:100073006E006875616E67006875690068756E006B
:1000830068756F006F6E67006F750075616E007540
:100093006900756E00756F0061202020006975008E
:1000A30072007561007561690075616E6700756145
:1000B3006E67200069610069616E6700696F6E6732
:1000C30000756500760068616E67200068756100E1
:1000D300B0A2B0A100B0A5B0A7B0A6B0A3B0A4B021
:1000E300A8B0A9B0ABB0AAB0ACB0AEB0AFB0AD00E1
:1000F300B0B2B0B1B0B0B0B3B0B6B0B4B0B8B0B7DE
:10010300B0B500B0B9B0BAB0BB00B0BCB0BDB0BE02
:10011300B0BFB0C0B0C1B0C2B0C4B0C300B0CBB008
:10012300CDB0C8B0C7B0C9B0C5B0CCB0C6B0CAB006
:10013300CEB0CFB0D1B0D0B0D3B0D6B0D5B0D4005C
:10014300B0D7B0D9B0DBB0D8B0DAB0DCB0DDB0DE58
:1001530000B0E2B0E0B0E3B0E4B0DFB0E1B0E5B0EE
:10016300E6B0ECB0EBB0E9B0E7B0E8B0EDB0EA0070
:10017300B0EEB0EFB0F0B0F3B0F1B0F2B0F6B0F86B
:10018300B0F4B0F9B0F5B0F700B0FCB0FAB0FBB022
:10019300FDB1A2B1A6B1A5B1A3B1A4B1A8B1A7B154
:1001A300AAB1ABB1A9B1ACB0FEB1A1C6D900B1B08F
:1001B300B1ADB1AFB1AEB1B1B1B4B1B7B1B8B1B323
:1001C300B1B5B1B6B1BBB1B9B1BAB1B200B1BCB19D
:1001D300BEB1BDB1BFBABB00B1C0B1C1B1C2B1C341
:1001E300B1C5B1C400B1C6B1C7B1C8B1CBB1CAB111
:1001F300C9B1D2B1D8B1CFB1D5B1D3B1D1B1DDB1DC
:10020300D0B1D6B1D4B1CDB1D7B1CCB1CEB1DAB1D1
:10021300DCB1DB00B1DFB1E0B1DEB1E1B1E2B1E508
:10022300B1E3B1E4B1E9B1E6B1E7B1E800B1EBB1F3
:10023300EAB1ECB1ED00B1EFB1EEB1F0B1F100B163
:10024300F6B1F2B1F3B1F5B1F4B1F700B1F9B1F828
:10025300B1FBB1FCB1FAB1FEB1FDB2A2B2A100B2E1
:10026300A6B2A8B2A3B2A7B2B1B2A4B2A5B2AEB2BB
:10027300B5B2AFB2B4B2AAB2ACB2B0B2A9B2B3B271
:10028300ABB2ADB2B2B2B700B2B9B2B8B2B6B2BBEA
:10029300B2BCB2BDB2C0B2BFB2BAB2BE00B2C1004C
:1002A300B2C2B2C5B2C4B2C6B2C3B2C9B2CAB2C78D
:1002B300B2C8B2CBB2CC00B2CEB2CDB2D0B2CFB212
:1002C300D1B2D2B2D300B2D6B2D7B2D4B2D5B2D8A9
:1002D30000B2D9B2DAB2DCB2DBB2DD00B2E1B2E035
:1002E300B2DEB2E2B2DF00B2E3B2E4D4F800B2E6C7
:1002F300B2E5B2E9B2E7B2E8B2EBB2ECB2EAB2ED20
:10030300B2EFB2EEC9B200B2F0B2F1B2F200B2F49F
:10031300B2F3B2F7B2F6B2F8B2F5B2FAB2F9B2FB8F
:10032300B2FC00B2FDB2FEB3A6B3A2B3A5B3A3B3AE
:10033300A7B3A1B3A8B3A9B3ABB3AA00B3ADB3AE8C
:10034300B3ACB3B2B3AFB3B0B3B1B3B3B3B4B4C27A
:1003530000B3B5B3B6B3B9B3B8B3B7B3BA00B3BBAD
:10036300B3BEB3BCB3C0B3C1B3BDB3C2B3BFB3C4F5
:10037300B3C300B3C6B3C5B3C9B3CAB3D0B3CFB362
:10038300C7B3CBB3CDB3CCB3CEB3C8B3D1B3D2B36E
:10039300D300B3D4B3D5B3DAB3D8B3DBB3D9B3D6BD
:1003A300B3DFB3DEB3DDB3DCB3E2B3E0B3E3B3E1B6
:1003B30000B3E4B3E5B3E6B3E7B3E800B3E9B3F0FE
:1003C300B3F1B3EBB3EEB3EDB3EFB3EAB3ECB3F323
:1003D300B3F2B3F400B3F6B3F5B3FDB3F8B3FCB3C0
:1003E300FAB3FBB3F7B3F9B4A1B4A2B3FEB4A6B4A2
:1003F300A4B4A5B4A3D0F300B4A700B4A8B4A9B41B
:10040300ABB4ACB4AAB4ADB4AE00B4B3B4AFB4B08F
:10041300B4B2B4B400B4B5B4B6B4B9B4B7B4B800F4
:10042300B4BAB4BBB4BFB4BDB4BEB4BCB4C000B4FE
:10043300C100B4C3B4CAB4C4B4C9B4C8B4C7B4C59E
:10044300B4C6B4CBB4CEB4CCB4CD00B4D1B4D3B46D
:10045300D2B4D0B4CFB4D400B4D500B4D6B4D9B4E4
:10046300D7B4D800B4DAB4DCB4DB00B4DEB4DFB4A0
:10047300DDB4E0B4E3B4E1B4E2B4E400B4E5B4E67B
:10048300B4E700B4EAB4E8B4E9B4ECB4EBB4ED0017
:10049300B4EEB4EFB4F0B4F1B4F2B4F300B4F4B422
:1004A300F5B4F6B4FAB4F8B4FDB5A1B4F9B4FBB439
:1004B300FCB4FEB4F700B5A4B5A5B5A3B5A2B5A623
:1004C300B5A8B5A7B5A9B5ABB5AEB5AFB5ACB5AD28
:1004D300B5B0B5AA00B5B1B5B2B5B3B5B4B5B5004D
:1004E300B5B6B5BCB5BAB5B9B5B7B5BBB5B8B5BD95
:1004F300B5BFB5C1B5C0B5BE00B5C3B5C2B5C400BF
:10050300B5C6B5C7B5C5B5C8B5CBB5CAB5C900B5C8
:10051300CDB5CCB5CEB5D2B5CFB5D0B5D3B5D1B5B4
:10052300D5B5D7B5D6B5D8B5DCB5DBB5DDB5DAB558
:10053300DEB5D900B5E0B5E1B5DFB5E4B5E3B5E2C5
:10054300B5E7B5E8B5E9B5EAB5E6B5EBB5EDB5ECB4
:10055300B5EEB5E500B5F3B5F0B5F2B5EFB5F1B568
:10056300F5B5F6B5F400B5F9B5F8B5FCB5FDB5FECE
:10057300B5FAB5FB00B6A1B6A3B6A2B6A4B6A5B6A6
:10058300A6B6A9B6A8B6A700B6AA00B6ABB6ACB6CF
:10059300ADB6AEB6AFB6B3B6B1B6B2B6B0B6B400DA
:1005A300B6BCB6B5B6B7B6B6B6B8B6B9B6BAB6BBD4
:1005B30000B6BDB6BEB6C1B6BFB6C0B6C2B6C4B647
:1005C300C3B6CAB6C5B6C7B6C8B6C9B6C600B6CBF3
:1005D300B6CCB6CEB6CFB6D0B6CD00B6D1B6D3B6BE
:1005E300D4B6D200B6D6B6D8B6D5B6D7B6DCB6DB57
:1005F300B6D9B6DD00B6E0B6DFB6E1B6DEB6E4B630
:10060300E2B6E3B6E7B6E9B6E6B6E8B6E500B6EFB6
:10061300B6EDB6F0B6EBB6ECB6EAB6EEB6F2B6F3B6
:10062300B6F1B6F6B6F5B6F400B6F700B6F9B6F815
:10063300B6FBB6FAB6FDB6FCB6FEB7A100B7A2B7D5
:10064300A6B7A5B7A3B7A7B7A4B7A8B7A900B7AB71
:10065300B7ACB7ADB7AAB7B2B7AFB7B0B7B3B7AE6A
:10066300B7B1B7B4B7B5B7B8B7BAB7B9B7B6B7B71D
:1006730000B7BDB7BBB7BCB7C0B7C1B7BFB7BEB78D
:10068300C2B7C3B7C4B7C500B7C9B7C7B7C8B7C63A
:10069300B7CAB7CBB7CCB7CDB7CFB7D0B7CEB7D133
:1006A30000B7D6B7D4B7D7B7D2B7D5B7D3B7D8B7BC
:1006B300DAB7D9B7DBB7DDB7DCB7DEB7DFB7E00052
:1006C300B7E1B7E7B7E3B7E2B7E8B7E5B7E9B7E646
:1006D300B7E4B7EBB7EAB7ECB7EDB7EFB7EE00B7F0
:1006E300F000B7F100B7F2B7F4B7F5B7F3B8A5B7B1
:1006F300FCB7F6B7F7B7FEB7FDB7FAB8A1B8A2B71C
:10070300FBB8A4B7F9B8A3B7F8B8A7B8A6B8AEB8FA
:10071300ABB8A9B8AAB8A8B8ADB8AFB8B8B8BCB8A0
:10072300B6B8BEB8BAB8BDB8C0B8B7B8B4B8B0B840
:10073300B1B8B5B8BBB8B3B8BFB8B9B8B200B8C2EE
:10074300B8C100B8C3B8C4B8C6B8C7B8C8B8C5003C
:10075300B8C9B8CAB8CBB8CEB8CCB8CDB8D1B8CF71
:10076300B8D2B8D0B8D300B8D4B8D5B8DAB8D9B8F5
:10077300D8B8D7B8D6B8DBB8DC00B8DEB8E1B8DF94
:10078300B8E0B8DDB8E2B8E3B8E5B8E4B8E600B875
:10079300EAB8EDB8E7B8ECB8EBB8EEB8E9B8E8B842
:1007A300F3B8EFB8F1B8F0B8F4B8F6B8F7B8F5BFE6
:1007B300A900B8F800B8F9B8FA00B8FCB8FDB8FB5E
:1007C300B8FEB9A1B9A2B9A300B9A4B9ADB9ABB97F
:1007D300A6B9A5B9A9B9ACB9A7B9AAB9A8B9AEB907
:1007E300AFB9B0B9B2B9B100B9B4B9B5B9B3B9B762
:1007F300B9B6B9B9B9BAB9B8B9BB00B9C0B9BEB914
:10080300C3B9C2B9C1B9BDB9BCB9BFB9C5B9C8B912
:10081300C9B9C7B9C6B9C4B9CCB9CAB9CBB9CD007E
:10082300B9CFB9CEB9D0B9D1B9D2B9D300B9D4B946
:10083300D5B9D600B9D8B9DBB9D9B9DAB9D7B9DDE1
:10084300B9DCB9E1B9DFB9E0B9DE00B9E2B9E3B9BE
:10085300E400B9E9B9E7B9EAB9E6B9EBB9E8B9E54A
:10086300B9ECB9EEB9EFB9EDB9F4B9F1B9F3B9F03F
:10087300B9F200B9F5B9F6B9F700B9F9B9F8B9FAA7
:10088300B9FBB9FCB9FD00B8F2B9FE00BAA2BAA12E
:10089300BAA3BAA5BAA7BAA6BAA400BAA8BAA9BAFB
:1008A300ACBAAABAAFBAADBAAEBAABBAB1BAB0BA09
:1008B300BABAB9BAB5BAB7BAB4BAB8BAB6BAB3BAB1
:1008C300B200BABCBABDD0D000BAC1BAC0BABFBABE
:1008D300BEBAC3BAC2BAC5BAC6BAC400BAC7BAC8DE
:1008E300BACCBACFBACEBACDBAD3BAD2BACBBAC9C6
:1008F300BAD4BAD0BACABAD8BAD6BAD5BAD700BA5D
:10090300DABAD900BADBBADCBADDBADE00BAE0BAC9
:10091300DFBAE3BAE1BAE200BAE4BAE5BAE6BAEB9F
:10092300BAECBAEABAE9BAE7BAE800BAEEBAEDBA8B
:10093300EFBAF0BAF3BAF1BAF200BAF5BAF4BAF60A
:10094300BBA1BAFCBAFABAF8BAFEBAF9BAF7BAFD59
:10095300BAFBBBA2BBA3BBA5BBA7BBA4BBA600BBE7
:10096300A8BBAABBA9BBACBBABBBAFBBAEBBADBB50
:10097300B000BBB3BBB2BBB4BBB1BBB500BBB6BB72
:10098300B9BBB7BBB8BBBABBC3BBC2BBBDBBBBBBAD
:10099300C1BBBCBBC0BBBEBBBF00BBC4BBC5BBCA2A
:1009A300BBCBBBC6BBCCBBCDBBC8BBC7BBC9BBD01A
:1009B300BBCEBBD1BBCF00BBD2BBD6BBD3BBD4BB9F
:1009C300D5BBD8BBD7BBDABBDCBBE3BBE1BBE4BB6A
:1009D300E6BBE5BBE2BBDFBBDEBBE0BBDDBBD9BB3C
:1009E300DB00BBE8BBE7BBE9BBEBBBEABBEC00BB93
:1009F300EDBBEEBBF0BBEFBBF2BBF5BBF1BBF6BB94
:100A0300F3BBF400BCA5BBF7BCA2BBF8BBFABCA10B
:100A1300BCA6BCA3BCA7BBFDBBF9BCA8BCA9BBFBC4
:100A2300BBFEBBFCBCA4BCB0BCAABCB3BCB6BCB4D0
:100A3300BCABBCB1BCB2BCACBCAFBCB5BCADBCAE5A
:100A4300BCB8BCBABCB7BCB9BCC6BCC7BCBFBCCDC8
:100A5300BCCBBCC9BCBCBCCABCC1BCBEBCC8BCC38F
:100A6300BCCCBCC5BCC4BCC2BCC0BCBBBCBDBDE56E
:100A730000BCD3BCD0BCD1BCCFBCD2BCCEBCD4BCDC
:100A8300D5BCD7BCD6BCD8BCDBBCDDBCDCBCD9BCBC
:100A9300DEBCDAD0AE00BCE9BCE2BCE1BCDFBCE446
:100AA300BCE7BCE8BCE6BCE0BCE3BCEABCE5BCF02C
:100AB300BCF3BCEDBCEBBCF1BCF5BCF4BCECBCEFD3
:100AC300BCF2BCEEBCFBBCFEBDA8BDA4BDA3BCF682
:100AD300BCFABDA1BDA7BDA2BDA5BDA6BCF9BCF80E
:100AE300BCFCBCFD00BDADBDAABDABBDACBDA9BDCD
:100AF300AEBDB2BDB1BDB0BDAFBDB3BDB5BDB4003C
:100B0300BDBBBDBCBDBFBDBDBDBEBDBABDB7BDB91F
:100B1300BDB6BDB8BDC7BDC6BDCABDC8BDC3BDC5D5
:100B2300BDC2BDC1BDCBBDC9BDD0BDCEBDCFBDCC8A
:100B3300BDD1BDCDBEF5BDC000BDD7BDD4BDD3BDF8
:100B4300D5BDD2BDD6BDDABDD9BDDCBDE0BDE1BDED
:100B5300DDBDDEBDD8BDDFBDE3BDE2BDE9BDE4BDA6
:100B6300E6BDECBDE7BDEABDEBBDE800BDEDBDF103
:100B7300BDEFBDF0BDF2BDEEBDF3BDF6BDF4BDF7F7
:100B8300BDF5BEA1BEA2BDFCBDF8BDFABDFEBDFD57
:100B9300BDFBBDF900BEA9BEADBEA5BEA3BEAABE28
:100BA300A7BEA6BEACBEA4BEABBEA8BEAEBEB1BE03
:100BB300B0BEAFBEBBBEB6BEB7BEBABEB9BEB4BE94
:100BC300B8BEB3BEB2BEB500BEBCBEBD00BEC0BEE5
:100BD300BFBEBEBEC5BEC3BEC4BEC1BEC2BEC6BE10
:100BE300C9BECABECCBECEBEC7BEC8BECDBECB007C
:100BF300BED3BED0BED1BED4BED2BECFBED6BDDB69
:100C0300BED5BED7BEDABED9BED8BEE4BEDEBEDC1C
:100C1300BEDFBEE6BEE3BEE7BEE5BEDDBEE0BEE2CE
:100C2300BEDBBEE100BEEABEE8BEE9BEEDBEEBBE82
:100C3300EEBEEC00BEEFBEF6BEF7BEF1BEF8BEF3ED
:100C4300BEF2BEF4BEF000BEFCBEFDBEF9BEFBBEEE
:100C5300FABFA1BFA4BEFEBFA3BFA5BFA200BFA78B
:100C6300BFA6BFA800BFAABFABBFADBFAEBFAC009E
:100C7300BCF7BFAFBFB1BFB0BFB2BFB3BFB400BF5C
:100C8300B5BFB6BFB7BFB8BFBABFB9BFBB00BFBC64
:100C9300BFBDBFBEBFBF00BFC0BFC1BFC2BFC6BF16
:100CA300C3BFC5BFC4BFC7BFC8BFC9BFCABFCBBF10
:100CB300CCBFCDBFCE00BFCFBFD1BFD2BFD000BF4F
:100CC300D4BFD300BFD5BFD7BFD6BFD800BFD9BF0E
:100CD300DABFDBBFDC00BFDDBFDEBFDFBFE0BFE2EB
:100CE300BFE3BFE100BFE4BFE5BFE6BFE8BFE70086
:100CF300BFE9BFECBFEBBFEA00BFEDBFEE00BFEF44
:100D0300BFF0BFF1BFF6BFF5BFF3BFF2BFF400BF43
:100D1300F7BFF9BFF8BFFABFFCBFFBBFFDBFFEC003
:100D2300A2C0A3C0A100C0A4C0A5C0A6C0A700C004
:100D3300A9C0A8C0ABC0AA00C0ACC0ADC0B2C0AE11
:100D4300C0B0C0AFC0B100C0B4C0B3C0B500C0BC78
:100D5300C0B9C0B8C0B7C0BBC0B6C0BEC0BDC0BAC2
:100D6300C0C0C0BFC0C2C0C1C0C3C0C400C0C9C02E
:100D7300C7C0C8C0C5C0C6C0CAC0CB00C0CCC0CDE8
:100D8300C0CEC0CFC0D0C0D1C0D4C0D3C0D200C0A9
:100D9300D6C0D5C1CB00C0D7C0D8C0DDC0DAC0D95A
:100DA300C0DCC0DFC0E1C0E0C0DBC0DE00C0E2C029
:100DB300E3C0E400C0E5C0E6C0EAC0EBC0F2C0E7B0
:100DC300C0ECC1A7C0E8C0E9C0F1C0EEC0EFC1A844
:100DD300C0EDC0F0C1A6C0FAC0F7C1A2C0F4C0F60E
:100DE300C0FBC0F8C1A4C0FDC1A5C0FEC0F3C0F5DF
:100DF300C0F9C1A3C0FCC1A100C1ACC1B1C1AFC1A5
:100E0300B0C1ABC1AAC1AEC1ADC1B2C1B3C1B7C15B
:100E1300B6C1B5C1B400C1A9C1BCC1B9C1BAC1B8D9
:100E2300C1BBC1BDC1C1C1C2C1BEC1C0C1BF00C17F
:100E3300CAC1C9C1C6C1C4C1C5C1C8C1CEC1C3C16C
:100E4300C7C1CDC1CFC1CC00C1D0C1D3C1D2C1D4E0
:100E5300C1D100C1DAC1D6C1D9C1DCC1D5C1D8C1A4
:100E6300D7C1DBC1DDC1DFC1DEC1E000C1E6C1E93D
:100E7300C1EBC1E1C1E8C1E5C1EAC1E7C1E2C1E338
:100E8300C1E4C1ECC1EEC1ED00C1EFC1F5C1F7C1D1
:100E9300F4C1F0C1F2C1F3C1F1C1F6C1F8C1F90067
:100EA300C1FAC1FCC1FDC1FBC2A1C1FEC2A4C2A261
:100EB300C2A300C2A6C2A5C2A7C2A8C2AAC2A90051
:100EC300C2B6C2ACC2AEC2ABC2AFC2ADC2B1C2B295
:100ED300C2B0C2B3C2BDC2BCC2B8C2B9C2BBC2B542
:100EE300C2B7C2BEC2BAC2B400C2CFC2CDC2CEC2A2
:100EF300D0C2D1C2D200C2D3C2D400C2D5C2D8C2DA
:100F0300D7C2D9C2DAC2D6C2DB00C2DEC2DCC2DFBC
:100F1300C2E0C2E1C2E2C2DDC2E3C2E5C2E7C2E6A9
:100F2300C2E400C2CBC2BFC2C0C2C2C2C3C2C1C23A
:100F3300C5C2C6C2C4C2C9C2C7C2CAC2CCC2C80023
:100F4300C2E8C2E9C2EDC2EAC2EBC2ECC2EEC2F031
:100F5300C2EF00C2F1C2F2C2F5C2F3C2F4C2F6009C
:100F6300C2F9C2F8C2F7C2FAC2FCC3A1C2FDC2FEF3
:100F7300C2FB00C3A6C3A2C3A4C3A3C3A7C3A50044
:100F8300C3A8C3ABC3ACC3A9C3AAC3AEC3ADC3AFEA
:100F9300C3B0C3B3C3B1C3B200C3B400C3BBC3B60E
:100FA300C3B5C3BCC3B7C3BDC3BAC3B8C3B9C3BF57
:100FB300C3C0C3BEC3C3C3C1C3C4C3C200C3C5C3C9
:100FC300C6C3C700C3C8C3CBC3CAC3CDC3C9C3CC7D
:100FD300C3CFC3CE00C3D6C3D4C3D5C3D1C3D3C336
:100FE300D2C3D7C3D0C3DAC3D9C3D8C3DCC3DDC329
:100FF300DB00C3DFC3E0C3DEC3E2C3E3C3E4C3E197
:10100300C3E5C3E600C3E7C3E8C3E9C3EBC3ECC36B
:10101300EAC3EEC3ED00C3F0C3EF00C3F1C3F3C3F0
:10102300F2C3F6C3F5C3F400C3FBC3F7C3F9C3FAB2
:10103300C3F8C3FC00C3FD00BAD1C3FEC4A1C4A35B
:10104300C4A4C4A6C4A5C4A2C4A7C4A8C4A9C4AD47
:10105300C4B0C4AAC4AFC4AEC4ABC4AC00C4B2C4AD
:10106300B1C4B300C4B8C4B6C4B5C4B7C4B4C4BE71
:10107300C4BFC4C1C4BCC4B9C4BBC4C0C4BDC4BA66
:10108300C4C200C4C3C4C4C4C7C4C9C4C8C4C6C4D6
:10109300C500C4CBC4CCC4CAC4CEC4CD00C4D0C460
:1010A300CFC4D100C4D200C4D3C4D5C4D4C4D6C41D
:1010B300D700C4D800C4DAC4D900C4DB00C4DC0040
:1010C300C4DDC4E1C4E0C4DFC4DEC4E3C4E2C4E6F7
:1010D300C4E4C4E7C4E500C4E9C4EAC4EDC4ECC491
:1010E300EBC4EEC4E800C4EFC4F000C4F1C4F200E2
:1010F300C4F3C4F9C4F4C4F6C4F7C4F8C4F500C413
:10110300FA00C4FEC5A1C4FCC4FBC4FDC5A200C54E
:10111300A3C5A4C5A6C5A500C5A9C5A8C5A7C5AA35
:1011230000C5ABC5ACC5AD00C5AF00C5B1C5B0000A
:10113300C5B2C5B5C5B3C5B400C5AE00C5B600C517
:10114300B7C5B9C5B8C5BBC5BCC5BAC5BD00C5BF64
:10115300C5BEC5C0B0D2C5C3C5C1C5C200C5C4C51F
:10116300C7C5C5C5C6C5C9C5C800C5CBC5CAC5CCD5
:10117300C5CDC5D0C5D1C5CEC5CF00C5D2C5D3C594
:10118300D4C5D5C5D600C5D7C5D9C5D8C5DAC5DB3D
:10119300C5DCC5DD00C5DEC5DFC5E3C5E0C5E2C509
:1011A300E1C5E6C5E5C5E400C5E7C5E800C5EAC590
:1011B300E9C5EBC5F3C5EDC5EFC5F0C5EEC5F4C58F
:1011C300ECC5F1C5F2C5F5C5F600B1D9C5FAC5F749
:1011D300C5FBC5F8C5FCC5F9C6A4C5FEC6A3C6A113
:1011E300C5FDC6A2C6A5C6A6C6A8C6A7C6A900C6EB
:1011F300ACC6ABC6AAC6AD00C6AFC6AEC6B0C6B116
:1012030000C6B2C6B300C6B4C6B6C6B5C6B7C6B87E
:1012130000C6B9C6BDC6C0C6BEC6BAC6BBC6C1C671
:10122300BFC6BC00C6C2C6C3C6C4C6C5C6C8C6C63A
:10123300C6C9C6C700C6CA00B8ACC6CDC6CBC6CCE5
:10124300C6CEC6D0C6CFC6D1C6D3C6D4C6D2C6D6DE
:10125300C6D5C6D7C6D800C6DFC6E3C6DEC6E2C655
:10126300E0C6DCC6DDC6DAC6DBC6E1C6EEC6EBC643
:10127300E4C6E6C6E7C6EDC6EAC6E9C6E8C6EFC6F3
:10128300E5C6ECC6F2C6F3C6F1C6F4C6F0C6F8C6A8
:10129300FDC6F9C6FAC6FBC6FCC6F5C6F6C6F70018
:1012A300C6FEC7A1C7A200C7A7C7AAC7A4C7A8C726
:1012B300A5C7A3C7A6C7ABC7A9C7B0C7AEC7AFC7A4
:1012C300ACC7B1C7ADC7B3C7B2C7B4C7B7C7B5C754
:1012D300B6C7B800C7BAC7BCC7B9C7BBC7BFC7BDC6
:1012E300C7BEC7C000C7C4C7C3C7C2C7C1C7C7C774
:1012F300C8C7C5C7C6C7C9C7CEC7CDC7CFC7CCC761
:10130300CBC7CA00C7D0C7D1C7D2C7D3C7D400C7BA
:10131300D7C7D6C7D5C7DBC7D8C7D9C7DDC7DAC7CD
:10132300DCC7DEC7DF00C7E0C7E2C7E1C7E3C7E446
:10133300C7E5C7E9C7E7C7E8C7E6C7EAC7EBC7EC2E
:1013430000C7EEC7ED00C7F0C7F1C7EFC7F4C7F397
:10135300C7F6C7F5C7F200C7F8C7FAC7FDC7FCC78A
:10136300F9C7FBC7F7C7FEC8A1C8A2C8A3C8A5C8C9
:10137300A400C8A6C8ABC8A8C8AAC8ADC8ACC8A9A9
:10138300C8A7C8AEC8B0C8AF00C8B2C8B1C8B3C850
:10139300B4C8B8C8B7C8B5C8B600C8B9C8BA00C8D1
:1013A300BBC8BCC8BDC8BE00C8BFC8C2C8C0C8C1CE
:1013B300C8C300C8C4C8C5C8C600C8C7C8C800C811
:1013C300CBC8CAC8C9C8CCC8D0C8CFC8CEC8D2C871
:1013D300D1C8CD00C8D3C8D400C8D500C8D6C8DE8C
:1013E300C8D7C8D9C8DDC8DCC8D8C8DBC8DAC8DFE5
:1013F30000C8E1C8E0C8E200C8E7C8E3C8E5C8E63A
:10140300C8E4C8EAC8E9C8E8C8EBC8EC00C8EEC835
:10141300ED00C8EFC8F1C8F000C8F2C8F300C8F483
:10142300C8F500C8F6C8F7C8F800C8FBC8F9C8FA79
:10143300C8FC00C8FDC8FEC9A1C9A200C9A3C9A4AC
:10144300C9A500C9A6C9A7C9A8C9A900C9ABC9AC80
:10145300C9AA00C9AD00C9AE00C9B1C9B3C9B4C9ED
:10146300B0C9AFC9B5C9B6C9B7CFC300C9B8C9B93F
:1014730000C9BDC9BEC9BCC9C0C9BAC9BFC9C1C9F0
:10148300C2C9C7C9BBC9C8C9C6C9C9C9C3C9C5C9EE
:10149300C4D5A400C9CBC9CCC9CAC9D1C9CEC9CD89
:1014A300C9CFC9D000C9D3C9D2C9D5C9D4C9D7C92D
:1014B300D6C9D8C9D9C9DBC9DCC9DA00C9DDC9DED7
:1014C300C9E0C9DFC9E1C9E8C9E7C9E4C9E6C9E2B6
:1014D300C9E5C9E300C9EAC9ECC9EDC9EBC9F0C95B
:1014E300EFC9E9C9EEC9F1C9F2C9F3C9F4C9F6C92B
:1014F300F5C9F8C9F7CAB200C9FDC9FAC9F9C9FCE7
:10150300CAA4C9FBC9FECAA1CAA5CAA2CAA300B379
:10151300D7CAACCAA7CAA6CAADCAABCAA9CAA8CAFF
:10152300AACAAECAAFCAB1CAB6CAB5CAB0CAB4CAE1
:10153300B3CAB7CAB8CAB9CABCCABBCABACABFCA8D
:10154300CFCAC0CACBCAD0CABECABDCAC2CACCCA15
:10155300C6CAD3CAD4CACECAD2CAD1CAC3CAC7CAD0
:10156300C1CACACAC5CACDCAC8CAC4CAC9CBC600B9
:10157300CAD5CAD6CAD8CAD7CAD9CADCCADECADB50
:10158300CADACADD00CAE9CAE3CAE5CAE0CAE2CADE
:10159300E1CAE7CAE8CAE6CAE4CADFCAEBCAEACACA
:1015A300ECCAEECAF2CAF0CAF3CAF1CAEDCAEFCA6C
:1015B300F5CAF9CAF8CAF6CAF7CAFACBA1CAFCCA6D
:1015C300FDCAFBCAFECAF400CBA2CBA300CBA5CBBA
:1015D300A4CBA6CBA700CBA9CBA800CBABCBAACBE4
:1015E300AC00CBADCBAECBB0CBAF00CBB1CBB3CBA1
:1015F300B4CBB200CBB5CBB8CBB7CBB600CBBFCB5C
:10160300BECBBDCBBCCBB9CBBBCBBACBC0CBC8CB92
:10161300C4CBC2CBC5CBC7CBC3CBC100CBC9CBCB10
:10162300CBCACBCFCBCECBD0CBCDCBCC00CBD4CBBB
:10163300D1CBD2CBD300CBD5CBD6CBD7CBDFCBE063
:10164300CBD8CBD9CBDACBDCCBDDCBDB00CBE1CB3F
:10165300E2CBE300CBE4CBE7CBE5CBE6CBE8CBEACD
:10166300CBEECBECCBE9CBEDCBEB00CBEFCBF0CBA5
:10167300F100CBF4CBF3CBF2CBF5CBF9CBF7CBF635
:10168300CBF800CBFDCBFBCBFCCBFACBFECCA1CC78
:10169300A2CCA4CCA300CCA5CCA8CCA7CCA6CCAB85
:1016A300CCADCCACCCA9CCAA00CCAECCB0CCAFCC1E
:1016B300B2CCB1CCB3CCB8CCB5CCB7CCB6CCB4CC23
:1016C300B9CCBBCCBACCBECCBFCCBDCCBC00CCC09F
:1016D300CCC6CCC3CCC4CCC1CCC2CCC5CCC7CCC883
:1016E300CCCACCC9CCCCCCCB00CCCECCD0CCCDCC02
:1016F300CFCCD3CCD2CCD5CCD4CCD1CCD6CCD700B8
:10170300CCD800CCDBCCDACCDCCCD900CCDECCDD45
:10171300CCE0CCDFCCE4CCE1CCE2CCE3CCE5CCEB4D
:10172300CCEACCE9CCE8CCE6CCE700CCECCCEDCCF5
:10173300EFCCF1CCF0CCEECCF3CCF200B5F7CCF49B
:10174300CCF5CCF6CCF7CCF800CCF9CCFACCFB003A
:10175300CCFCCDA1CCFDCCFECDA2CDA4CDA5CDA3FB
:10176300CDA6CDA700CDA8CDACCDAECDA9CDADCD69
:10177300AFCDAACDABCDB3CDB1CDB0CDB2CDB4004D
:10178300CDB5CDB7CDB6CDB800CDB9CDBACDBBCDE6
:10179300BCCDBDCDBFCDBECDC0CDC1CDC2CDC300AF
:1017A300CDC4CDC500CDC6CDC7CDC8CDCBCDC9CD5C
:1017B300CA00B6DACDCCCDCDCDCE00CDD0CDCFCDF8
:1017C300D1CDD4CDD3CDD5CDD2CDD7CDD6CDD8CD0A
:1017D300D900CDDBCDDECDDACDDDCDDCCDDFCDE087
:1017E30000CDE1CDE200CDE4CDE5CDE3CDE8CDEA1A
:1017F300CDE6CDE7CDE9CDF0CDECCDEDCDF1CDEF1F
:10180300CDEECDEBCDF2CDF300CDF4CDF6CDF5CDD0
:10181300F8CDF9CDF7CDFDCDFCCDFACDFB00CEA3B0
:10182300CDFECEA2CEA1CEAACEA4CEA7CEA5CEA6C5
:10183300CEA8CEA9CEACCEABCEB0CEB1CEB2CEB3C7
:10184300CEADCEAFCEAECEC0CEB4CEBBCEB6CEB77F
:10185300CEB8CEBECEBDCEB9CEBCCEB5CEBFCEBA3F
:1018630000CEC2CEC1CEC4CEC6CEC5CEC3CEC7CEA9
:10187300C9CEC8CECA00CECCCECBCECD00CECECE36
:10188300D0CED1CECFCED2CED6CED4CED5CED3001F
:10189300CEDACEDBCED8CED7CEDDCEDCCED9CEDE01
:1018A300CEE3CEE2CEE1CEDFCEE0CEE5CEE7CEE9AB
:1018B300CEEBCEE4CEEACEE6CEE8CEF0CEF1CEEC61
:1018C300CEEFCEF3CEF2CEEECEED00CFA6CFABCEA3
:1018D300F7CEFCCFA3CEF4CEF6CEF9CFA2CEFECF79
:1018E300A4CFA7CFA9CEF8CEFACFACCFA1CFAACEA3
:1018F300FDCFA8CEF5CEFBCFA5CFB0CFAFCFAECF28
:10190300B1CFADCFB4CFB2CFB7CFB5CFB8CFB6008D
:10191300CFBACFB9CFBBCFC0CFBFCFC1CFBECFBD63
:10192300CFBCCFC2CFC5CFC400CFB3CFC9CFC8CFF1
:10193300CBCFC6CFC7CFCACFD0CFD2CFCDCFCCCFCF
:10194300D1CFCFCFCECFD3CFD4CFD5CFD8CFD6CF84
:10195300DFCFDECFDCCFDDCFDACFDBCFD7CFD90000
:10196300CFE7CFE0CFE3CFE1CFE6CFE4CFE5CFE2E0
:10197300CFEACFE9CFE8CFEDCFECCFEBCFF2CFEF8C
:10198300CFEECFF3CFF1CFF000CFFCCFFBCFF4CF2F
:10199300F5CFFACFF6CFF9CFFDD0A1CFFED0A2D0AD
:1019A300A4CFF8D0A7D0A3D0A6D0A500D0A9D0A803
:1019B300D0AAD0ABD0ADD0B0D0B2D0B1D0B3D0AF2D
:1019C300D0ACD0B4D0B9D0BAD0B6D0BCD0B5D0BBDF
:1019D300D0B8D0B700D0C4D0C3D0BED0C1D0C0D04F
:1019E300BFD0C2D0BDD0C5D0C600D0CBD0C7D0CA1F
:1019F300D0C9D0C8D0CCD0CFD0CED0CDD0D1D0D3F9
:101A0300D0D5D0D2D0D400D0D7D0D6D0D9D0DAD078
:101A1300D8D0DBD0DC00CBDED0DDD0DED0DFD0E031
:101A2300D0E3D0E5D0E4D0E2D0E100D0E7D0EBD0F2
:101A3300E9D0EAD0E8D0E6D0ECD0EDD0F1D0F2D0C6
:101A4300F0D0F4D0F7D0F8D0EFD0F6D0F5D0EED375
:101A5300F500D0F9D0FBD0FAD0FED0FCD0FDD1A157
:101A6300D1A2D1A4D1A300CFF7D1A5D1A6D1A8D11A
:101A7300A7D1A9D1AA00D1ABD1ACD1B0D1B2D1AE4B
:101A8300D1B1D1AFD1ADD1B5D1B6D1B4D1B8D1B730
:101A9300D1B300D1BED1B9D1BDD1BAD1BBD1BCD1A3
:101AA300C0D1BFD1C1D1C2D1C4D1C3D1C6D1C5D197
:101AB300C7D1C800D1CAD1CCD1CDD1C9D1CBD1D313
:101AC300D1CFD1D4D1D2D1D8D1D7D1D0D1CED1D6F3
:101AD300D1D1D1D5D1D9D1DCD1DAD1DBD1DDD1E1AD
:101AE300D1E5D1E2D1E4D1E7D1DED1E9D1E8D1DF4B
:101AF300D1E6D1E3D1E000D1EBD1EAD1EDD1ECD104
:101B0300EFD1F2D1F4D1EED1F0D1F1D1F3D1F6D1BD
:101B1300F8D1F5D1F7D1F9D1FA00BDC4D1FDD1FC8B
:101B2300D1FBD2A2D2A6D2A4D2A5D2A1D2A3D1FE56
:101B3300D2A7D2A8D2A9D2AAD2ABD4BF00D2ACD258
:101B4300ADD2AFD2AED2B2D2B1D2B0D2B5D2B6D27A
:101B5300B7D2B3D2B9D2B4D2BAD2B800D2BBD2C1FF
:101B6300D2C2D2BDD2C0D2BFD2BCD2BED2C7D2C4DF
:101B7300D2CAD2CBD2CCD2C8D2C6D2C5D2C3D2C992
:101B8300D2CDD2D2D2D1D2D4D2D3D2CFD2D0D2CE3E
:101B9300D2E5D2DAD2E4D2D5D2E9D2E0D2D9D2ECAC
:101BA300D2DBD2D6D2EBD2D8D2D7D2EFD2E8D2DFA1
:101BB300D2E6D2EAD2EED2DDD2E2D2E7D2DED2E16F
:101BC300D2E3D2EDD2DC00D2F2D2F5D2F6D2F0D209
:101BD300F1D2F4D2F3D2F7D2FAD2F9D2F8D2FCD2BC
:101BE300FDD2FBD2FED3A100D3A6D3A2D3A4D3A705
:101BF300D3A3D3A5D3ADD3AFD3ABD3A8D3A9D3AA00
:101C0300D3ACD3AED3B1D3B0D3B3D3B200D3B40038
:101C1300D3B6D3B5D3B8D3B9D3BAD3B7D3C0D3BD5F
:101C2300D3BED3C2D3BFD3C1D3BCD3BBD3C300D3DF
:101C3300C5D3C7D3C4D3C6D3C8D3C9D3CCD3CAD3CC
:101C4300CDD3CBD3CED3D1D3D0D3CFD3D6D3D2D37B
:101C5300D7D3D3D3D5D3D400D3D8D3D9D3E5D3DAF9
:101C6300D3E8D3E0D3DBD3E3D3E1D3E9D3E6D3E7BC
:101C7300D3E4D3E2D3DED3DCD3DDD3DFD3EBD3EEB4
:101C8300D3ECD3F0D3EAD3EDD3EFD3F1D4A6D3F38C
:101C9300D3FDD3F4D3FCD3F8D4A1D4A4D3F2D3FB90
:101CA300D3F7D4A2D3F9D4A3D3F6D3FAD3FED4A5CE
:101CB30000D4A9D4A7D4A8D4AAD4B1D4B0D4ABD4D3
:101CC300ADD4B2D4ACD4AED4B5D4B4D4B3D4AFD4ED
:101CD300B6D4B7D4B9D4BAD4B800D4BBD4BCD4C264
:101CE300D4C0D4C3D4C4D4BED4C1D4BD00D4C6D408
:101CF300C8D4C7D4C5D4CAD4C9D4D0D4CBD4CED4F1
:101D0300CDD4CFD4CC00D4D1D4D3D4D2D5A600D47F
:101D1300D6D4D5D4D4D4D7D4D8D4D9D4DAD7D00040
:101D2300D4DBD4DCD4DDD4DE00D4DFD4E0D4E100D2
:101D3300D4E2D4E3D4E4D4E7D4E6D4E9D4E8D4E5D4
:101D4300D4EED4EDD4ECD4EBD4EFD4EA00D4F2D473
:101D5300F1D4F3D4F000D4F400D4F500D4F6D4F7DE
:101D6300D4F900D4FBD4FCD4FAD4FDD4FED5A2D547
:101D7300A1D5A3D5A7D5A9D5A8D5A5D7F500D5AB0A
:101D8300D5AAD5ACB5D4D5ADD5AED5AF00D5B4D5E0
:101D9300B1D5B3D5B2D5B0D5B6D5B9D5B5D5B8D5F6
:101DA300B7D5BCD5BDD5BBD5BED5C0D5BFD5BA007B
:101DB300B3A4D5C5D5C2D5C3D5C4D5C1D5C7D5C69A
:101DC300D5C9D5CCD5CAD5C8D5CDD5CBD5CFD5CE0C
:101DD30000D5D0D5D1D5D2D5D3D5D9D5D7D5D4D58E
:101DE300D5D5D6D5D8D7A600D5DAD5DBD5DCD5DD84
:101DF300D5DED5DFD5E0D5E2D5E3D5E1D7C500D52E
:101E0300EAD5EBD5ECD5E4D5E6D5E8D5E5D5E7D5E8
:101E1300E9D5EFD5EDD5EED5F3D5F1D5F2D5F0D69D
:101E2300A100D5F9D5F7D5FAD5F5D5F8D5F6D5F47A
:101E3300D5FCD5FBD5FDD6A4D6A3D5FED6A200D618
:101E4300AED6A7D6ADD6A5D6A8D6A6D6AAD6AFD691
:101E5300ABD6ACD6A9D6B4D6B6D6B1D6B5D6B0D64F
:101E6300B2D6B3D6B9D6BBD6BCD6B7D6BDD6B8D6FE
:101E7300BAD6C1D6BED6C6D6C4D6CED6CBD6CAD689
:101E8300C5D6BFD6C8D6C2D6C0D6CCD6CFD6C7D66F
:101E9300CDD6C9D6C300D6D0D6D2D6D5D6D1D6D3F1
:101EA300D6D4D6D7D6D6D6D9D6DAD6D800D6DDD696
:101EB300DBD6DFD6DCD6DED6E0D6E1D6E2D6E3D675
:101EC300E4D6E6D6E7D6E5D6E800D6ECD6EFD6EAF2
:101ED300D6E9D6EED6EDD6EBD6F1D6F2D6F0D6F7D6
:101EE300D6F4D6F3D6F6D6F5D7A1D6FAD7A2D6FC32
:101EF300D7A4D6F9D7A3D6F8D6FBD6FED6FD00D7FE
:101F0300A500D7A700D7A8D7A9D7AAD7ABD7AD0025
:101F1300D7B1D7AFD7AED7B0D7B3D7B4B4B1D7B2A1
:101F230000D7B7D7B5D7B6D7B9D7BAD7B800D7BBC5
:101F3300D7BC00D7BFD7BED7BDD7C0D7C6D7C2D7A8
:101F4300C7D7C3D7C4D7C100D7CED7C8D7C9D7CB74
:101F5300D7CAD7CDD7CCD7D1D7D3D7CFD7D2D7D648
:101F6300D7D4D7D500D7DAD7DBD7D8D7D9D7D7D7D0
:101F7300DCD7DD00D7DED7DFD7E0D7E100D7E2D764
:101F8300E3D7E4D7E5D7E7D7E8D7E9D7E600D7AC77
:101F9300D7EBD7EA00D7ECD7EED7EFD7ED00D7F0E2
:101FA300D7F100D7F2D7F3D7F4D7F7D7F8D7F9D7C4
:101FB300F60000FF0003FF00D3FF0004FF00D8FF7B
:101FC3000006FF00F3FF0008FF0106FF000BFF01FF
:101FD3000DFF000DFF0120FF000FFF0143FF001263
:101FE300FF0154FF0015FF0173FF0019FF018CFF70
:101FF300001CFF01B1FF001FFF01D0FF0022FF0102
:10200300DBFF0004FF01E8FF0026FF0217FF002AA1
:10201300FF0230FF002EFF0239FF0031FF0242FFB3
:102023000034FF024FFF000BFF0262FF0038FF0284
:102033008BFF000DFF02A0FF000FFF02A3FF0012A2
:10204300FF02BAFF0015FF02C9FF0019FF02D4FF08
:10205300003AFF02DFFF0022FF02EAFF003CFF021B
:10206300F1FF003FFF030AFF0043FF0311FF004797
:10207300FF0326FF004CFF033FFF0050FF0354FF05
:102083000053FF0361FF0057FF0376FF005CFF036C
:1020930095FF005FFF03B4FF0064FF03BFFF006809
:1020A300FF03D8FF006BFF03FBFF0070FF03FEFF7E
:1020B3000075FF040DFF007BFF0418FF007FFF0482
:1020C30023FF0083FF0432FF0004FF0435FF008772
:1020D300FF044EFF008BFF045BFF0038FF045EFF2D
:1020E300008EFF0467FF0092FF046EFF0095FF045C
:1020F3007FFF0098FF0486FF009BFF0493FF000F00
:10210300FF04A0FF0012FF04B9FF0015FF04D8FF6E
:102113000019FF04E3FF003AFF04FCFF0022FF0560
:1021230003FF0004FF0512FF0026FF0537FF002A07
:10213300FF0558FF002EFF0569FF0034FF0578FFF8
:1021430000A0FF058BFF0087FF058EFF008BFF05B7
:10215300A3FF0038FF05B4FF008EFF05D1FF0092F7
:10216300FF05DEFF0095FF05E7FF0098FF05F8FF79
:102173000003FF0611FF0006FF062CFF00A3FF0666
:102183002FFF000DFF0640FF0012FF0651FF001551
:10219300FF0674FF001CFF068BFF001FFF06A4FF52
:1021A3000022FF06C3FF000BFF06E2FF008BFF06C2
:1021B300E5FF0038FF06E8FF000DFF0741FF000FB2
:1021C300FF0746FF0012FF0753FF0015FF076AFFD3
:1021D3000019FF077DFF003AFF0792FF001CFF076E
:1021E300B5FF001FFF0753FF0022FF07BDFF008756
:1021F300FF07CCFF008BFF07EBFF0038FF07FEFF55
:1022030000A5FF0823FF00A8FF0830FF008EFF088A
:1022130037FF00ACFF084EFF0092FF0855FF009503
:10222300FF0876FF0098FF087DFF000DFF088AFF77
:10223300000FFF088FFF0012FF089EFF0015FF0825
:10224300C5FF0019FF08CCFF003AFF08DFFF001CA1
:10225300FF0902FF001FFF0907FF0022FF0910FF0C
:102263000087FF091BFF008BFF092EFF0038FF09C2
:102273003DFF00A5FF0962FF00A8FF0975FF008E5F
:10228300FF0980FF00B1FF099DFF0092FF09BAFF1C
:102293000095FF09E5FF0098FF09F2FF0003FF1F08
:1022A300B5FF0004FF0A07FF00B7FF0A74FF00260B
:1022B300FF0A99FF00BAFF0AE8FF002AFF0B03FF9A
:1022C300002EFF0B3CFF0031FF0B6FFF0034FF0BB1
:1022D30098FF00BFFF0BCBFF00A0FF0BD0FF003820
:1022E300FF0BF3FF008EFF0C28FF00C4FF0C37FF2A
:1022F3000095FF0C4AFF000DFF0C61FF000FFF0C60
:1023030068FF0012FF0C73FF0015FF0C82FF00191A
:10231300FF0C91FF003AFF0C9AFF001FFF0CB9FF5F
:102323000022FF0CC2FF0087FF0CC7FF008BFF0CCE
:10233300D0FF0038FF0CD9FF00A5FF0CE8FF00A871
:10234300FF0CF3FF008EFF0CFCFF00ACFF0D01FF41
:102353000092FF0D12FF0095FF0D29FF0098FF0D5E
:1023630032FF000DFF0D3BFF000FFF0D4AFF001270
:10237300FF0D51FF0015FF0D70FF0019FF0D7FFFCB
:10238300003AFF0D92FF001CFF0D99FF0022FF0D85
:10239300B0FF0004FF0DB7FF0026FF0DFCFF00BADE
:1023A300FF0E19FF002AFF0E32FF002EFF0E4BFF18
:1023B3000031FF0E56FF0034FF0E6FFF00A0FF0E2B
:1023C3008CFF0087FF0EA3FF008BFF0EB6FF0038C4
:1023D300FF0EC3FF008EFF0EECFF00C4FF0EF9FFDC
:1023E3000095FF0EFEFF0098FF0F0DFF00C7FF0FC4
:1023F30026FF000DFF0F43FF000FFF0F56FF0012D4
:10240300FF0F63FF0015FF0F76FF0019FF0F83FF18
:10241300003AFF0F9CFF001CFF0F9FFF001FFF0FE1
:10242300C0FF0022FF0FC7FF0004FF0FD8FF0026E5
:10243300FF0FF5FF002AFF1008FF002EFF1019FF02
:102443000031FF101EFF0034FF102BFF00A0FF1010
:1024530038FF000BFF103BFF008BFF1060FF0038BD
:10246300FF1067FF000DFF1086FF000FFF1095FFA1
:102473000012FF10A0FF0015FF10A7FF0019FF10A7
:10248300AAFF003AFF10B5FF001CFF10B8FF001FA2
:10249300FF10BDFF0022FF10C0FF0004FF10C3FFA9
:1024A3000026FF10DAFF00BAFF10E9FF002AFF1031
:1024B300EEFF002EFF10F3FF0031FF1102FF003487
:1024C300FF1105FF00A0FF1112FF0087FF111BFF83
:1024D3000038FF1124FF008EFF112BFF00C4FF11F2
:1024E3002EFF0098FF1133FF00C7FF113CFF0003CD
:1024F300FF113FFF0038FF1142FF000DFF1151FF95
:10250300000FFF1160FF0012FF116DFF0015FF1197
:102513007EFF0019FF1189FF001CFF1198FF001FA8
:10252300FF11ABFF0022FF11B0FF0004FF11CDFF2D
:102533000026FF11F2FF002AFF11FBFF002EFF12FE
:1025430004FF0031FF1209FF0034FF1214FF000BD8
:10255300FF1227FF008BFF1238FF0038FF123BFFEB
:102563000004FF125AFF00B7FF12A3FF0026FF1259
:10257300AAFF00BAFF12D7FF002AFF12E8FF002EBE
:10258300FF1307FF0031FF1312FF0034FF1329FF6E
:1025930000BFFF1344FF00A0FF1349FF0038FF13E0
:1025A3005AFF008EFF1375FF00C4FF138CFF0095C5
:1025B300FF139DFF0012FF13A2FF0015FF13ABFFD4
:1025C3000019FF13B6FF003AFF13BDFF001FFF13EF
:1025D300C2FF0022FF13D7FF0004FF13DCFF0087B5
:1025E300FF13DFFF008BFF13F4FF0038FF13FBFF24
:1025F300008EFF1410FF0092FF1415FF0095FF14C7
:102603001CFF0098FF1421FF000DFF1426FF000F8D
:10261300FF142DFF0012FF1436FF0015FF143FFFB8
:102623000019FF1446FF003AFF144FFF001FFF1469
:1026330056FF0022FF1459FF003CFF145CFF003FCC
:10264300FF146FFF0043FF1474FF00C9FF1497FFCB
:10265300004CFF14A8FF0050FF14BFFF0053FF14EA
:10266300D8FF0057FF14FBFF005CFF1512FF006447
:10267300FF1573FF0068FF1588FF00CFFF15CBFF21
:10268300006BFF15D0FF0070FF15D9FF0075FF1514
:10269300DEFF007BFF15E5FF007FFF15EEFF0083E4
:1026A300FF15F7FF0004FF1600FF0087FF161FFF4B
:1026B300008BFF1630FF0038FF1639FF008EFF1620
:1026C30050FF0092FF1657FF0095FF166EFF00980C
:1026D300FF1675FF000DFF1686FF000FFF1699FF0B
:1026E3000012FF16ACFF0015FF16D1FF0019FF16ED
:1026F300ECFF003AFF1703FF0022FF1706FF000459
:10270300FF170FFF0026FF172EFF002AFF173FFFBB
:10271300002EFF174CFF0034FF1753FF0087FF17EE
:1027230068FF008BFF1783FF0038FF178CFF008EB5
:10273300FF17A3FF0092FF17A8FF0095FF17B5FF30
:102743000098FF17BEFF0003FF1FB5FF0003FF1F25
:10275300B5FF000DFF17D5FF000FFF17E4FF0012B1
:10276300FF17E9FF0015FF180CFF001CFF1821FFDE
:10277300001FFF1864FF0022FF1879FF000BFF18EA
:1027830080FF0038FF1893FF0004FF18CEFF00B747
:10279300FF1913FF0026FF198CFF00BAFF1963FF0F
:1027A300002AFF198CFF002EFF19AFFF0031FF191C
:1027B300D8FF0034FF19EDFF00BFFF1A0AFF00A086
:1027C300FF1A19FF0038FF1A2EFF008EFF1A55FF5C
:1027D30000C4FF1A6AFF0095FF1A79FF000DFF1A64
:1027E30096FF0012FF1AB7FF0015FF1AFAFF001930
:1027F300FF1B1DFF003AFF1B40FF0004FF1B5FFF91
:102803000031FF1BCAFF0034FF1BEBFF000BFF1C53
:1028130010FF0087FF1C13FF008BFF1C32FF0038E3
:10282300FF1C5BFF008EFF1CB4FF00C4FF1CDDFF19
:102833000095FF1CF0FF000DFF1D09FF000FFF1D9A
:1028430012FF0012FF1D23FF0015FF1D2CFF0019AF
:10285300FF1D33FF003AFF1D50FF001CFF1D59FFF2
:10286300001FFF1D5CFF0022FF1D5FFF003CFF1DDB
:1028730066FF003FFF1D81FF0043FF1D90FF0047E0
:10288300FF1DB3FF004CFF1DD4FF0050FF1DEBFFE6
:102893000053FF1E02FF0057FF1E25FF005CFF1EB3
:1028A30042FF005FFF1E99FF0064FF1EB0FF006838
:1028B300FF1ECDFF00CFFF1F02FF006BFF1F05FFB1
:1028C3000070FF1F08FF0075FF1F13FF007BFF1F32
:1028D30024FF007FFF1F31FF0083FF1F36FF00042B
:1028E300FF1F4BFF0087FF1F68FF008BFF1F77FF52
:1028F3000038FF1F80FF008EFF1F91FF0092FF1F14
:1029030098FF0095FF1FA1FF0098FF1FA6FF00037C
:03291300FF1FB5EE
:1030C6002036221FB61FD4203420FA2172218421F3
:1030D600BA222C229E22A422F8236423F4246624F6
:1030E600F024FC256225B6260A26D62748274E2731
:0930F60054278A27DE283829102E
:062E6D008B588A59895AB6
:102E7300AB58AA59A95A1231278F62AB58AA59A93C
:102E83005A122D68FFEF70077BFF7A0079032275D2
:102E93006100C3E5626480F8E5616480985023AB08
:102EA30058AA59A95AAF61EF3395E0FEE92FF9EA21
:102EB3003EFA122D68FFEF4420FFEF122DAE05619D
:102EC30080D0AB58AA59A95A122D68FFEFB46907ED
:102ED3007BFF7A00790322AB58AA59A95A122D68AD
:102EE300FFEFB475077BFF7A00790322AB58AA5929
:102EF300A95A122D68FFEFB476077BFF7A00790396
:102F030022AB58AA59A95A122D68FFEF25E0246075
:102F1300F8E6FE08E6FFAA06A9077BFF8B5B8A5C3F
:102F2300895DAB58AA59A95A122D68FFEF25E024F1
:102F330062F8E6FE08E6FFAA06A9077BFF8B5E8A16
:102F43005F89607401255AF55AE43559F559AB5E2A
:102F5300AA5FA960C003C002C001AB5BAA5CA95D04
:102F6300C3D082D083D0E0E99582EA958350697516
:102F73006100C3E5626480F8E5616480985036AB14
:102F83005BAA5CA95D122DC0AF61EF3395E0FE8FA4
:102F9300828E83122D81FFAB58AA59A95AAE61EED6
:102FA300FD3395E0FC8D828C83122D81FEEEB507F7
:102FB30004056180BDE561B56210AB5BAA5CA95DE8
:102FC300758203758300122DE0227406255DF55D7D
:0E2FD300E4355CF55C022F517BFF7A00790338
:012FE10022CD
:03000000022FE2EA
:0C2FE200787FE4F6D8FD7581620230298A
:102C7200E709F608DFFA8046E709F208DFFA803E44
:102C820088828C83E709F0A3DFFA8032E309F60831
:102C9200DFFA8078E309F208DFFA807088828C8399
:102CA200E309F0A3DFFA806489828A83E0A3F6084D
:102CB200DFFA805889828A83E0A3F208DFFA804C27
:102CC20080D280FA80C680D4806980F280338010FE
:102CD20080A680EA809A80A880DA80E280CA803367
:102CE20089828A83ECFAE493A3C8C582C8CCC583DF
:102CF200CCF0A3C8C582C8CCC583CCDFE9DEE780AF
:102D02000D89828A83E493A3F608DFF9ECFAA9F02D
:102D1200EDFB2289828A83ECFAE0A3C8C582C8CC83
:102D2200C583CCF0A3C8C582C8CCC583CCDFEADE9C
:102D3200E880DB89828A83E493A3F208DFF980CCFE
:102D420088F0EF60010E4E60C388F0ED2402B404F7
:102D52000050B9F582EB2402B4040050AF2323459E
:062D62008223902CC273D5
:102D6800BB010689828A83E0225002E722BBFE0269
:092D7800E32289828A83E493229C
:102D8100BB010CE58229F582E5833AF583E0225007
:102D910006E92582F8E622BBFE06E92582F8E22251
:0D2DA100E58229F582E5833AF583E493226B
:102DAE00BB010689828A83F0225002F722BBFE0104
:022DBE00F322FE
:102DC000BB010789828A83022E295005E9F8022E69
:102DD00010BBFE05E9F8022E3289828A83022E3B5F
:102DE000BB010DE58229F582E5833AF583022E29A0
:102DF0005007E92582F8022E10BBFE07E92582F86C
:102E0000022E32E58229F582E5833AF583022E3BD4
:10291600E517240BF8E60517227808300702780B2E
:10292600E475F001122E19022D682000EB7F2ED2DD
:10293600008018EF540F2490D43440D4FF30040B99
:10294600EF24BFB41A0050032461FFE51860021596
:1029560018051BE51B7002051A30070D7808E4758B
:10296600F001122E19EF022DAE0231007403D207C8
:102976008003E4C207F5178B088A09890AE4F5186B
:10298600F51AF51BE51860077F2012295180F575A9
:1029960019FFC201C200C202C203C205C206C208B2
:1029A60012291FFF700D3007057F00122962AF1B29
:1029B600AE1A22B4255FC2D5C20412291FFF24D045
:1029C600B40A00501A75F00A781830D50508B6FF13
:1029D6000106C6A426F620D5047002D20380D924A7
:1029E600CFB41A00EF5004C2E5D204022B62D20122
:1029F60080C6D20080C0D20280BCD2D580BAD205B1
:102A060080B47F201229512002077401B5180040B6
:102A1600F1122916FF12295102298AD208D20680FC
:102A260095122916FB122916FA122916F94A4B7025
:102A36000679337A2C7BFF20022EE518602A7E0069
:102A46008E82758300122D8160060EEE651970F078
:102A5600C2D5EBC0E0EAC0E0E9C0E0EE122BA9D097
:102A6600E0F9D0E0FAD0E0FB122D68FF60AAEBC0D7
:102A7600E0EAC0E0E9C0E0122951D0E02401F9D033
:102A8600E03400FAD0E0FBE5190460DCD519D98002
:102A9600877BFF7A2B79A5D202809C7910800279F8
:102AA60008C206C2088008D2D5790A8004790AC20B
:102AB600D5E519047002F519E4FAFDFEFF12291690
:102AC600FC7B08200113122916FD7B1030000A1228
:102AD6002916FE122916FF7B20EC3382D592D5509B
:102AE60013C3E43000069FFFE49EFEE42001039D2D
:102AF600FDE49CFCE4CBF8C201EC700CCFCECDCC4F
:102B0600E824F8F870F38017C3EF33FFEE33FEEDD9
:102B160033FDEC33FCEB33FB994002FB0FD8E9EBBA
:102B2600300105F8D0E0C448B201C0E00AEC4D4ED1
:102B36004F78207B0070C2EAB5190040BCC0E01295
:102B46002BABD0F0D0E0200104C4C0E0C4B201C079
:102B5600F012293AD0F0D5F0EB02298A122E472A34
:102B660027532AA15829F84C29F4422AA54F2AAD01
:0F2B7600442AAD492A0D432AB3552A97462A9778
:102B8500452A97472C535029FC2D2A002E2A232B02
:102B95002A04232A21202C3C2A29BC4800002A1B70
:102BA5003F3F3F00790AA2D5200314300509B9102B
:102BB500020404B9080104A2D5200602500104202C
:102BC50002689202B518005034C0E07F2030031926
:102BD5007F30A20272067205500F122C02C202C289
:102BE50006C205C2087F30800F300503E9C0E01238
:102BF5002951300503D0E0F9D0E0B518CC300517E0
:102C05007F30B9100C1229517F583004077F788026
:102C150003B908031229513002057F2D0229517F7E
:102C2500202008F87F2B2006F322920280CF286E01
:102C3500756C6C2900D2011229163001F8C2017891
:102C45001830D50108F60229BC2D504349581229E0
:102C5500162403B405004001E4902C4E931229423A
:0D2C6500743A122942D203751804022AA104
:10312700E4FFFE122D68600C0FEF70010E09E970C5
:05313700F20A80EF2206
:102FEE0002306EE493A3F8E493A34003F68001F25B
:102FFE0008DFF48029E493A3F85407240CC8C333E4
:10300E00C4540F4420C8834004F456800146F6DFB2
:10301E00E4800B01020408102040809030C6E47E4C
:10302E00019360BCA3FF543F30E509541FFEE493A7
:10303E00A360010ECF54C025E060A840B8E493A36E
:10304E00FAE493A3F8E493A3C8C582C8CAC583CA99
:10305E00F0A3C8C582C8CAC583CADFE9DEE780BE51
:0130FF0000D0
:092E1000E6FB08E6FA08E6F922E7
:102E1900FAE6FB0808E6F925F0F618E6CA3AF622BA
:092E2900E0FBA3E0FAA3E0F922AA
:092E3200E2FB08E2FA08E2F922D1
:0C2E3B00E493FB740193FA740293F922F3
:102E4700D083D082F8E4937012740193700DA3A31A
:102E570093F8740193F5828883E47374029368602E
:062E6700EFA3A3A380DF2E
:10310000EFB40A07740D12310B740A309811A899A4
:10311000B8130CC2983098FDA899C298B811F6302F
:0731200099FDC299F5992207
:00000001FF
